:100000000C9464010C9481010C9481010C94810185
:100010000C9481010C9481010C9481010C94810158
:100020000C9481010C9481010C94FD1D0C94CF1E45
:100030000C9404190C9481010C9481010C9481019D
:100040000C9481010C9481010C9481010C94810128
:100050000C9481010C948C190C9481010C948101F5
:100060000C9481010C9493010C9481010C94F40183
:100070000C9481010C9481010C9481010C948101F8
:100080000C9481010C9481010C9481010C948101E8
:100090000C9481010C9481010C9481010C948101D8
:1000A0000C9481010C9481010C948101A604A60496
:1000B000D204D2043A055805700670066305FC05A3
:1000C0000D060D063C1F631F5B20631F5B20AF1FE7
:1000D000D21F5B2029203820290035001E001F0078
:1000E0002000210022002B0014001A000800150037
:1000F00017004B00E00004001600070009000A008A
:100100004C00E1001D001B00060019000500500016
:100110002F00E200E30065008A0076004A002C0010
:100120003A003B003C003D003E003F002E002D0009
:1001300027002600250024002300310013001200B0
:100140000C0018001C004E00280033000F000E00A9
:100150000D000B002A00E5003800370036001000C3
:1001600011004F003000E600E70065008B007600CC
:100170004D002C0041004000430042004500440077
:100180002603530070006C006900740065002000B5
:100190004B006500790062006F006100720064002E
:1001A0002000760033000000120357006800610051
:1001B0006C00650020004D006F000000040309047E
:1001C00009023B00020100A0FA090400000103013A
:1001D00001000921110100012240000705810308E7
:1001E00000010904010001030000000921110100C0
:1001F00001227B000705820320000112010002009A
:10020000000008EDFE95040300010200010501094C
:1002100002A10185020901A100050919012908159A
:100220000025019508750181020501093009311584
:1002300081257F95027508810609381581257F95EE
:100240000175088106050C0A38021581257F950184
:1002500075088106C0C005010980A1018503190147
:100260002AB700150126B700950175108100C00559
:100270000C0901A101850419012AA002150126A07B
:1002800002950175108100C005010906A10105074D
:1002900019E029E7150025019508750181029501EE
:1002A000750881010507190029FF150026FF009533
:1002B0000675088100050819012905950575019144
:1002C00002950175039101C011241FBECFEFDAE042
:1002D000DEBFCDBF11E0A0E0B1E0E0E4F2E402C097
:1002E00005900D92AA38B107D9F722E0AAE8B1E04B
:1002F00001C01D92A13AB207E1F70E9446130C9487
:100300001E210C940000F8949093CD008093CC00B3
:1003100082E08093C8008CED8093C90086E08093D2
:10032000CA00789408951F920F920FB60F9211246D
:100330002F933F938F939F93EF93FF938091C800E8
:100340002091C9009091CE008C71B9F421FF1AC0A0
:10035000913099F48AE692E090939401809393010E
:1003600086E090E090939601809395018CE891E06F
:1003700090939801809397012CC01092960110924F
:10038000950127C02091950130919601232B09F109
:10039000E0919301F0919401908380919301909169
:1003A000940101969093940180939301809195011B
:1003B0009091960101979093960180939501892BD6
:1003C00041F4E0919701F0919801309711F081E0AC
:1003D0008083FF91EF919F918F913F912F910F908B
:1003E0000FBE0F901F9018951F920F920FB60F928D
:1003F00011242F933F938F939F93EF93FF938091BB
:100400008F0190919001009719F12091C9002E7FE2
:100410002093C900E0918D01F0918E0120812093FD
:10042000CE0020918D0130918E012F5F3F4F309390
:100430008E0120938D0101979093900180938F01FD
:10044000892B31F4E0919101F091920181E0808358
:10045000FF91EF919F918F913F912F910F900FBE40
:100460000F901F901895E0918F01F0919001EF2B64
:10047000B9F49091C80095FF13C070938E016093FA
:100480008D015093900140938F01309392012093FE
:1004900091019091C90091609093C9008093CE0022
:1004A00080E090E0089580E090E00C9483010C944B
:1004B0005302282F80918C01882361F0AAE6B2E0D4
:1004C000E22FF92F9D91919392E0A037B907D1F7D0
:1004D00010928C010895EAE6F2E0DC012D91CD0145
:1004E0002193B2E0E037FB07C1F710928C012CE8B2
:1004F00031E046E050E06AE672E081E00C943302BD
:1005000081E0089581E008950C94820208950C948E
:1005100086021F93CF93DF9300D000D01F92CDB7F8
:10052000DEB749835A836B8330919A0189819A811E
:10053000311114C0662359F0222349F00E94AD08FE
:10054000182F682F89819A810E94560803C00E9443
:100550008108182F69817A81812F04C00E94AD081B
:1005600069817A810F900F900F900F900F90DF911B
:10057000CF911F910C94D60FFC01262F4081518101
:100580006281738184810C94890281E00895CF9304
:10059000DF93EC0160E00E94BC02BE01DF91CF91CD
:1005A0000C9487020C9422110C941E1108950E9441
:1005B00000070E94D6022FEF84E39CE02150804088
:1005C0009040E1F700C000000C94B2190F931F9304
:1005D000CF93DF938C0161E00E94BC02EC01B80173
:1005E0000E9484028823F1F1B801CE010E94C9174C
:1005F0008823C1F1B801CE010E94DD15882391F155
:10060000B801CE010E942517882361F1F80182818B
:10061000882309F1CB358DE5D807C1F050F4C11519
:10062000FCE5DF0781F0CF3DDC45A9F40E94E40D35
:1006300019C0CC35EDE5DE0761F0CD35DD4559F467
:100640000E94270D08C00E94D7020CC00E94300DE6
:1006500002C00E94330DC801DF91CF911F910F910D
:100660000C94800280E0DF91CF911F910F9108954B
:100670000E94E7180C9451030E9454030C94ED1847
:1006800008950C94400381E008950C944303089569
:10069000CF93C82F0E9441038C2F0E944503CF9116
:1006A000089580E00C9448030E9425180C94480398
:1006B0000E94251890919901891721F08093990142
:1006C0000C9448030895CF93DF93CDB7DEB72B97F3
:1006D0000FB6F894DEBF0FBECDBF4F835887698732
:1006E0007A878B8761110E94730C9E012F5F3F4FA9
:1006F00086E0F90111928A95E9F785E0FE013796C7
:10070000D90101900D928A95E1F789819A814C81F6
:100710005D81452B31F09F3F31F491E08F3F19F41B
:1007200003C091E001C090E090FF09C049815A8167
:100730006B817C818D819E810E94940B05C0C901D3
:100740000E94C5028111F2CF2B960FB6F894DEBF3E
:100750000FBECDBFDF91CF910895FC0180819181C3
:100760000E94EF080895CF93882309F450C0C82F42
:100770008CEF8C0F813AD0F46C2F80910201909114
:1007800003010E948918882349F06C2F809102018F
:10079000909103010E94C1180E94950C6C2F8091CA
:1007A0000201909103010E94BF180CC080E28C0FDF
:1007B000883058F4C77081E001C0880FCA95EAF705
:1007C0000E94560CCF910C94950CEBE5EC0FE330A6
:1007D00040F4F0E0E85BFE4F808190E0CF910C9414
:1007E0005118E8E5EC0FE73150F4F0E0EE0FFF1F91
:1007F000E65EFE4F80819181CF910C946718CD3ECB
:1008000030F08C2F0E94CB13CF910C949D14CF917C
:100810000895882389F19CEF980F913A40F4682F4E
:1008200080910201909103010E94C1180DC090E2D5
:10083000980F983058F4877091E001C0990F8A950D
:10084000EAF7892F0E945C0C0C94950C9BE5980F9D
:10085000933020F480E090E00C94511898E5980FC4
:10086000973120F480E090E00C9467188D3E20F0E2
:100870000E9426140C949D1408951F93CF93DF9328
:10088000182FEB010E94B303209741F08FE99FE0FE
:100890000197F1F700C000002197F6CF812FDF917B
:1008A000CF911F910C940904893319F060E070E036
:1008B00002C060E570E00C943D04882321F00E94A2
:1008C000560C0C94950C0895882321F00E945C0C22
:1008D0000C94950C0895CF92DF92EF92FF920F93B4
:1008E0001F93CF93DF937C01D62FC72FFC0112817A
:1008F000058102950F700E944C0C8823B9F01123DA
:10090000A9F08C2F807F803421F080E28D0F883019
:1009100068F08091750282FD09C082E00E94F50CAA
:100920000E944C0C91E0D82ED92601C0D12CCC2E9F
:10093000C2948FE0C8228C2D90E08C30910508F095
:10094000CFC1FC01EA5AFF4F0C94B5208C2F807F59
:10095000CF70882311F0C295C07F112399F0CC236A
:1009600009F4AAC180E28D0F883010F0D11104C0C3
:100970008C2F0E94560C03C08C2F0E94660C0E9484
:10098000950C9AC18D2F0E940904CC2309F4A8C1AB
:1009900080E28D0F883038F1DD2329F18C2F0E9401
:1009A0006C0C24C08C2F807FCF70803211F0C295E8
:1009B000C07FDD2319F0D130A1F13DC080917502D7
:1009C00082FF17C0112349F0CC2329F08C2F0E94FD
:1009D000560C0E94950C80E070C180E00E940904D2
:1009E000CC2309F47DC18C2F0E945C0C0E94950CD5
:1009F00077C1112371F0002341F0013031F40E94DE
:100A0000760C8C2B0E947E0C6BC10E94760C8C2B7A
:100A10001DC0002319F0013009F462C10E948B0C43
:100A200025C0112321F0063008F05AC10EC0053050
:100A300008F056C11BC0112361F0002331F0F7010B
:100A4000858180FF39C18F7085838C2F0E945D0462
:100A500047C1002359F0D93309F03FC1FFEF07EE3A
:100A600013E0F15000401040E1F735C18C2F0E9497
:100A7000640436C18C2F86958695837019F0813079
:100A800061F02EC1112321F08D2F9C2F937002C095
:100A900080E090E00E9451182BC1112321F08D2F8E
:100AA0009C2F937002C080E090E00E94671820C1E4
:100AB0008D2F112319F00E94CB1302C00E9426141F
:100AC0000E949D1415C18C2F837009F047C011112D
:100AD0000BC12D2F229526952770220F220F6D2FE7
:100AE0006F70862F90E0A0E0B0E0022E04C0880F67
:100AF000991FAA1FBB1F0A94D2F7D4FF10C04FE062
:100B000050E060E070E004C0440F551F661F771F7F
:100B10002A95D2F7409550956095709503C040E0B6
:100B200050E0BA01C695C695C3708A019B01082B97
:100B3000192B2A2B3B2BC901B801C23049F058F4BC
:100B4000C13019F00E946C07CFC00E945A07CCC078
:100B50000E947E07C9C00E945807C6C0112319F021
:100B60008C2F817001C08695882309F4BDC02D2F7C
:100B7000229526952770220F220F6D2F6F70862FDA
:100B800090E0A0E0B0E0022E04C0880F991FAA1FD9
:100B9000BB1F0A94D2F7D4FF10C04FE050E060E0D2
:100BA00070E004C0440F551F661F771F2A95D2F7C7
:100BB000409550956095709503C040E050E0BA01B3
:100BC000C695C695C3708A019B01082B192B2A2B49
:100BD0003B2BC901B801C23049F058F4C13019F0BB
:100BE0000E94310881C00E941F087EC00E944308F5
:100BF0007BC00E94920778C0CF70112339F08C2FF0
:100C00000E94B8078D2F0E945D046EC08D2F0E9438
:100C100064048C2F0E94D90767C0D23F21F128F4C9
:100C2000D03F41F0D13FC1F043C0D33F19F1D43F91
:100C300079F03EC0112341F0053008F051C08C2FEF
:100C40008F710E94FE074CC0063008F049C0F7CFF4
:100C50008091750282FF18C0112339F08C2F8F719B
:100C60000E94B8073DC01123C9F38C2F8F710E94D9
:100C7000D90736C0112329F08C2F8F710E94A3074A
:100C80002FC00E949E072CC0112349F0CF718C2FDA
:100C90000E94B80763E08C2F0E94DA0C21C081E02B
:100CA0000E94F50C0230E0F082E00E94F50C18C0C2
:100CB000112331F0002391F28D2F0E94B30310C055
:100CC000002399F2D93349F41FEF27EE33E0115096
:100CD00020403040E1F700C000008D2F0E94090441
:100CE00088EF8C0D843020F40E9425180E94480360
:100CF000DD20C9F00E94480C80FD15C0F70112826A
:100D00000E94420C0E94B807C7010E94B4060E94CC
:100D1000420CDF91CF911F910F91FF90EF90DF90E8
:100D2000CF900C94D907DF91CF911F910F91FF9035
:100D3000EF90DF90CF9008950F931F93CF93DF93A1
:100D4000EC01688179818A810E94FA088C010E94F5
:100D500055080E944607B801CE010E946B04DF913E
:100D6000CF911F910F910895CF93DF93EC0198815C
:100D700089812B813C81232B31F08F3F31F481E03D
:100D80009F3F19F403C081E001C080E080FD1DC0D9
:100D9000CE010E94E602811110C00E944C0C8823F3
:100DA000A1F08A81882389F08091750282FD0DC0AF
:100DB00082E0DF91CF910C94F50CCE010E949C064D
:100DC000CE01DF91CF910C94C702DF91CF910895AE
:100DD00080E090E00E94511880E090E00E94671847
:100DE0000E94730C0E94950C0E94CE150C949D14C9
:100DF00080910201909103010E94C3180C94E806AF
:100E00000E94630C0C94F80692959F70963079F0CE
:100E100010F4925001C09A50923068F4803F69F00B
:100E200018F4883E40F409C0843F29F406C0883E87
:100E300020F0813F11F080E0089581E00895FC01E9
:100E4000808191810E94EF080E9404070895CF934A
:100E5000DF9300D000D01F92CDB7DEB70F900F9078
:100E60000F900F900F90DF91CF910895CF93DF9364
:100E700000D000D000D0CDB7DEB726960FB6F894DC
:100E8000DEBF0FBECDBFDF91CF91089508950895C5
:100E90000C9447070C9448070E944A076093D601B8
:100EA0007093D7018093D8019093D9010C94E806F0
:100EB0000C944C070F931F930091D6011091D7010A
:100EC0002091D8013091D901602B712B822B932B6B
:100ED0001F910F910C944C070F931F930091D60113
:100EE0001091D7012091D8013091D901602371234D
:100EF000822393231F910F910C944C070F931F9300
:100F00000091D6011091D7012091D8013091D901DB
:100F100060277127822793271F910F910C944C070C
:100F20000C9447070E9490076093D2017093D301FD
:100F30008093D4019093D5010C94E80660E070E0B2
:100F4000CB010C9492070F931F9341E050E060E0B7
:100F500070E08A019B0104C0000F111F221F331F84
:100F60008A95D2F7C901B8011F910F910C9492078D
:100F70000F931F9341E050E060E070E004C0440F25
:100F8000551F661F771F8A95D2F78091D2019091E5
:100F9000D301A091D401B091D5018A019B01082B06
:100FA000192B2A2B3B2BC901B8011F910F910C94CF
:100FB00092070F931F9341E050E060E070E004C09F
:100FC000440F551F661F771F8A95D2F7409550959D
:100FD000609570958091D2019091D301A091D40138
:100FE000B091D5018A019B01082319232A233B23B1
:100FF000C901B8011F910F910C9492070F931F9391
:1010000041E050E060E070E004C0440F551F661FEF
:10101000771F8A95D2F78091D2019091D301A09148
:10102000D401B091D5018A019B01082719272A27ED
:101030003B27C901B8011F910F910C9492070F93A0
:101040001F930091D2011091D3012091D4013091CE
:10105000D501602B712B822B932B1F910F910C9438
:1010600092070F931F930091D2011091D301209109
:10107000D4013091D50160237123822393231F91E2
:101080000F910C9492070F931F930091D20110912E
:10109000D3012091D4013091D50160277127822797
:1010A00093271F910F910C949207089527E0929F28
:1010B000800D1124E82FE695E695E695877051E0BE
:1010C00001C0550F8A95EAF785E0E89FF0011124E9
:1010D000E556FE4F20E030E070E04081CB01022E6B
:1010E00002C0969587950A94E2F7817081958427CE
:1010F0008523842781932F5F3F4F2530310569F782
:10110000089527E0929F800D1124682F66956695BB
:101110006695982F977085E0689FB001112440E094
:1011200050E080E0FB01E40FF51FE556FE4F208103
:1011300030E0092E02C0369527950A94E2F7217017
:101140003327042E01C0220F0A94EAF7822B4F5F47
:101150005F4F4530510531F70895BF92CF92DF922E
:10116000EF92FF920F931F93CF93DF938C01C09068
:10117000D201D090D301E090D401F090D5018091BC
:10118000D6019091D701A091D801B091D901C82A78
:10119000D92AEA2AFB2ACFE1D0E0D701C6010C2EDA
:1011A00004C0B695A795979587950A94D2F780FDC8
:1011B00004C0219790F7B12C07C0BC2EB8018C2F2A
:1011C0000E94E90F0197A9F38B2DDF91CF911F9119
:1011D0000F91FF90EF90DF90CF90BF900895CF9345
:1011E000DF93EC010E94AD08BE010E94E90FDF9180
:1011F000CF9108951F93CF93DF93EB0190919A01C4
:10120000992321F0CB010E94EF0813C0882349F0F5
:10121000CB010E94AD08182F682FCE010E945608FE
:1012200004C0CB010E948108182FBE01812F0E94AB
:10123000E90FDF91CF911F9108951F93CF93DF9313
:10124000C091DA0116E08091DB01C81799F0D0E077
:101250001C9FF0011D9FF00D1124E452FE4F4081B0
:10126000518162817381848195810E943607219624
:10127000C770E9CFDF91CF911F91089540910C0283
:1012800050910D0260910E0270910F028091100238
:10129000909111020C943607EF92FF920F931F93D7
:1012A000CF93DF938091110282958F7009F065C012
:1012B00080910E02882309F460C08091DA01F090D9
:1012C000DB0110910C0200910D0260910F027091F0
:1012D000100291E01F3F09F090E0C0910001D09111
:1012E0000101292F96E0E92E8F1509F446C06115FA
:1012F000710521F00F3F21F030E003C031E001C063
:10130000322F90E030FD36C0E89EF001E99EF00DEE
:101310001124DF01A452BE4F11963C911197301356
:1013200029C03C91311326C012963C91129731117D
:1013300021C013964D915C911497461B570B4C1787
:101340005D07C0F4809111028F708061809311025B
:10135000EF51FE4F80818F70806180838CE092E03E
:101360000E94B406DF91CF911F910F91FF90EF90F3
:101370000C941D0901968770B7CFDF91CF911F9113
:101380000F91FF90EF9008959F92AF92BF92CF92EE
:10139000DF92EF92FF920F931F93CF93DF93CDB71E
:1013A000DEB761970FB6F894DEBF0FBECDBF8C01DC
:1013B00085E0F801DE011D9601900D928A95E1F716
:1013C000D8011296EC9090910C02E0910D022091C0
:1013D0000F02309110022115310531F0EF3F31F449
:1013E00081E09F3F19F403C081E001C080E0B82F85
:1013F000B1709B2E80FD47C1D8014C9111965C9134
:1014000011971396AD90BC9014978CE0C82E82E093
:10141000D82EF0900E02B501621B730B20910001D3
:1014200030910101FF2009F4D9C0809111026217A7
:10143000730708F095C0282F207F09F052C05E1373
:1014400013C0491311C0FE2CE1100EC08F708061D3
:10145000809311020E943E09C6010E94B406809149
:101460001102F80185834DC1AB2831F05F3F31F4A3
:1014700081E04F3F19F403C081E001C080E080FDAE
:1014800003C081E08E2502C080E090E0F82FF1706B
:10149000FF2E80FF1CC08091DA012091DB0136E035
:1014A000821709F40BC190E0389FF001399FF00DCD
:1014B0001124E452FE4F6181561306C06081461329
:1014C00003C06281E61203C001968770E9CFFE2C4B
:1014D000EE2009F416C180911102816080931102FF
:1014E00054C05E1306C0491304C0E11002C0F801E5
:1014F00099C0C8010E941F07882361F1EE2051F1B5
:1015000020911102822F82958F7090E0029774F0E3
:1015100080910C0290910D0298878F831986BB866B
:10152000AA862C87CE0107960E94B40686E0F801B1
:10153000ACE0B2E001900D928A95E1F70E944C096F
:101540000E943E090AC05E1711F1C8010E941F07E0
:1015500081112CC0C8010E94B406FF24F394D1C0AD
:10156000282F207F81F77A2DB98AA88A6E2D898944
:101570000E9427078CE092E00E94B40686E0D60124
:101580001D928A95E9F70E943E09F12CBAC04913D1
:10159000DCCFE110DACFF8018583C8010E94B406E0
:1015A00086E0D6011D928A95E9F7ABC0EE2091F254
:1015B00020911102822F82958F7090E002970CF497
:1015C000B5CF80910C0290910D029A8389831B8282
:1015D000BD82AC822E83CE010196A6CF621773071F
:1015E00008F044C0FE2CEE2009F4B4CF5E1330C0E6
:1015F00049132EC02091110220FD21C0822F829517
:101600008F70482F50E041155105C9F0F80125832E
:101610004F30510541F08F5F982F9295907F822F28
:101620008F70892B8583C8010E94B40686E0F8017B
:10163000ACE0B2E001900D928A95E1F73CC086E003
:10164000F801ACE0B2E001900D928A95E1F759C043
:10165000C8010E941F07811169CF8091110281602A
:1016600080931102C8010E94B4064BC07A2DB98A3A
:10167000A88A6E2D89890E94270786E0D6011D92CF
:101680008A95E9F718C0EE2009F464CFC8010E94DA
:101690001F07F82E882309F45DCF86E0F801ACE03F
:1016A000B2E001900D928A95E1F78CE092E00E9401
:1016B000AD030E944C090E943E0923C04D875E87FE
:1016C0008D859E850E94EF08292F22952F7022304C
:1016D00028F49F7039F0811105C00BC0243028F424
:1016E0009F7049F4805E883020F0C8010E94B406E3
:1016F0009F2CF92C06C0D80115969C91907F91F7EC
:10170000F8CF8F2D61960FB6F894DEBF0FBECDBF18
:10171000DF91CF911F910F91FF90EF90DF90CF90CD
:10172000BF90AF909F9008951F93CF93DF93CDB755
:10173000DEB72C970FB6F894DEBF0FBECDBF4F8338
:10174000588769877A878B879C87CE0107960E9486
:10175000C4098823D1F09F8188852A853B85232B66
:1017600031F08F3F31F481E09F3F19F403C081E0F5
:1017700001C080E080FD47C04F81588569857A852A
:101780008B859C850E9436073EC086E0FE01379619
:10179000DE01119601900D928A95E1F7FF81E885AF
:1017A0006A857B856115710531F0EF3F31F481E089
:1017B000FF3F19F403C081E001C080E080FD23C039
:1017C0002091DB0130E0C901019687709927409193
:1017D000DA0150E084179507F1F1F983EA837D83FC
:1017E0006C8396E0929FD001939FB00D1124A45278
:1017F000BE4FFE01319601900D929A95E1F78093CC
:10180000DB010E941D0916E08091DA019091DB0155
:10181000891771F1189FC001112484529E4F0E94B4
:10182000C409882329F1E091DA011E9FF0011124F7
:10183000E452FE4F408151816281738184819581A0
:101840000E9436078091DA0190E00196877099270F
:101850008093DA01D9CF0E9400071092DB01109229
:10186000DA01ECE0F2E086E0DF011D928A95E9F70B
:101870002C960FB6F894DEBF0FBECDBFDF91CF918F
:101880001F91089580911A028595859585950895F3
:1018900080911A028770089590911A02977081E0E2
:1018A00009F480E008958091250208959091250221
:1018B000892B809325020895809590912502892394
:1018C0008093250208951092250208959091240294
:1018D000892B809324020895809590912402892376
:1018E00080932402089510922402089580911B028F
:1018F000089508950C94790C0C947A0C90917502CB
:1019000092FD08C090911B02981721F080931B0252
:101910000C947C0C089580911B02882329F010926E
:101920001B0280E00C947C0C0895CF93DF93E09130
:101930000201F0910301809125028083E091020170
:10194000F0910301908180912402892B8083809102
:101950001B02882381F0E0910201F0910301908144
:10196000892B808380910201909103010E947D1850
:1019700081110E948B0CC0910201D091030148E0BB
:1019800050E062E172E0CE010E94CF20892B69F025
:1019900088E0FE01A2E1B2E001900D928A95E1F7A4
:1019A000CE01DF91CF910C943818DF91CF9108953B
:1019B0000C94790C9091750292FD10C098E0899F6B
:1019C00090011124262B20931A020E94B8078091BF
:1019D0001A028595859585950C94D80C0C94B807BA
:1019E00010921A0280E00C94D80C20911A02809573
:1019F000822380931A02982F977099F430E0482F31
:101A0000082E000C550B2417350759F090917502DC
:101A100092FD07C08595859585950E94D9070C9400
:101A2000F00C08959091750292FB222720F9281757
:101A300069F080FB92F99093750280917402909105
:101A400075020E94600D82E00C94F50C089580915F
:101A5000750282FB882780F991E089270C94120D8A
:101A600081E00C94120D80E00C94120D6FEF7FEF6B
:101A700080E090E00C94082180E090E00E94E42057
:101A800021E0893E9E4F09F020E0822F089582E0F8
:101A900090E00C94DC2083E090E00C94DC20CF9369
:101AA00084E090E00E94DC20C82F82E290E00E9457
:101AB000DC202C2F30E0A901582BCA01CF910895CA
:101AC000CF93C92F682F84E090E00E94EA206C2F0A
:101AD00082E290E0CF910C94EA20AB01BC018FE050
:101AE00090E00C94FC20AB01BC0183E190E00C94ED
:101AF000FC2060E070E0CB010C94730D60E070E0BE
:101B0000CB010E946D0D0C94790D69EE7EEF80E0A3
:101B100090E00E94082160E082E090E00E94EA20CC
:101B200060E083E090E00E94EA201092D6011092DB
:101B3000D7011092D8011092D90160E084E090E0C2
:101B40000E94EA2060E082E290E00E94EA2060E0E9
:101B500085E090E00E94EA2060E086E090E00E944C
:101B6000EA206FEF87E090E00E94EA2040E050E03A
:101B7000BA0188E090E00E94FC2060E08DE090E0F7
:101B80000E94EA2040E050E0BA0188E190E00E9423
:101B9000FC2060E087E190E00E94EA2040E050E015
:101BA000BA018CE190E00E94FC2060E070E080E2ED
:101BB00090E00E94082140E050E0BA0188E190E006
:101BC0000E94FC200C947E0D0C94850D682F8EE0F5
:101BD00090E00C94EA200E94711960933602709391
:101BE00037028093380290933902609332027093E7
:101BF00033028093340290933502089585B780684C
:101C000085BF85B7806885BF08950C94D712089565
:101C10000C94070E0C94070E0C940A0E0C94070EED
:101C20000C940E0E0C94070E0E94FE0D8EEC90E1AB
:101C30000E941B180E94120E0C94100E0E94080E97
:101C40000C94070E0E94E8100C9447030E945C1944
:101C50000E94C5100E94F1120E9428120E94220EBA
:101C60000E94DC150E94FB120C940C0E8F929F9226
:101C7000AF92BF92CF92DF92EF92FF920F931F939A
:101C8000CF93DF93CDB7DEB72A970FB6F894DEBFB8
:101C90000FBECDBF0E944C12982E81110E94EB0DF9
:101CA00086E2A82E82E0B82E00E010E0802E802F81
:101CB0000E940C11D82EF501C1905F01C826B1F425
:101CC0000F5F1F4F0C30110589F78FEF89838A83CF
:101CD0001B820E9465198160782F9D838C834981C6
:101CE0005A816B818D810E9463032FC080913A02DB
:101CF00081FD0E941211E12CFF24F3948C2D8F2181
:101D0000F1F00E94050E882399F0EE828F82DF2089
:101D100081E009F480E088870E9465198160782F4E
:101D20009A8789874E815F8168858A850E946303CF
:101D3000F801EA5DFD4F8081F826F08206C0E39449
:101D4000FF0CF7E0EF12DACFBBCF81E0911001C0BA
:101D500080E02A960FB6F894DEBF0FBECDBFDF91AC
:101D6000CF911F910F91FF90EF90DF90CF90BF9098
:101D7000AF909F908F9008950E94360E0E94D712C8
:101D80000E94BB140C945803CF93DF930E94EE0F74
:101D9000EC01811521E5920708F045C0811530E579
:101DA000930708F094C0883E910528F5803E910580
:101DB00008F0F8C0883A910570F4853A910508F06A
:101DC0007CC08130910509F475C008F4E8C004971F
:101DD00008F0E8C0E4C08F3B910508F0E0C0C85AA5
:101DE000D0E0CC0FDD1FC55BDE4F0990D881C02D40
:101DF000CE019464D8C0811540E2940758F481154F
:101E000051E0950708F0CEC08D3E910508F4C7C09B
:101E10009065C9C0C11580E4D80708F4C0C0DF7060
:101E2000CE01906AC0C0811525E59207A8F48115FE
:101E300034E5930708F095C0811543E5940708F051
:101E40007BC0811552E5950708F061C0D82FCC27DB
:101E5000CE01816F906AA7C0C11589E5D807A0F4AB
:101E6000C11528E5D20708F082C0C11536E5D307B1
:101E700008F095C08C2F0E9482108F7190E0D82FAF
:101E8000CC27CE0190628FC0C1154AE5D40708F473
:101E900074C0CE0190568115904208F080C08D2FFD
:101EA0008F710E948210DD27D0628F71AE01582B96
:101EB000CA0179C081E090E076C0C55AD0E0C75829
:101EC000DE4F8881C82FD0E0CE0190646CC074E0F2
:101ED000969587957A95E1F7282F23703C2F3370DC
:101EE00081E090E002C0880F991F3A95E2F79C6864
:101EF000AC01522B9A019C2F9F709695969550E2BB
:101F0000959FE0011124C9018C2B9D2B4CC083703F
:101F1000992721E030E002C0220F331F8A95E2F7B3
:101F20009C2F9695969580E2989FE0011124C22BF4
:101F3000D32BCE019C6837C08370992721E030E015
:101F400002C0220F331F8A95E2F79C2F9695969533
:101F500040E2949FE0011124C22BD32BCE019A685A
:101F600022C0D82FCC27CE01846F906A1CC0DC2FF2
:101F7000CC27CE01806F906A16C08C2F8F700E9484
:101F8000821094E0D695C7959A95E1F7CF70D0E08E
:101F9000DC2FCC27D0699E01282BC90104C080E02A
:101FA00090E001C0CE01DF91CF91089524E5829F9A
:101FB000C0011124FC0127E0729FE00DF11D1124E6
:101FC000E60FF11DEE0FFF1FE852FF4F8591949130
:101FD00008950E94D60F0E94C40E0895823891057C
:101FE00069F1B0F48133910509F46DC048F4893288
:101FF000910509F463C08A32910509F469C0089516
:102000008533910509F455C089339105B9F00895D8
:10201000833E910569F138F4803E9105B1F0823E2E
:10202000910509F10895863E9105A9F1873E910534
:10203000B9F1843E910509F064C023C02091740277
:1020400020FD4FC021FD4DC008958091740280FD98
:1020500044C08091750280FF44C08091740284FD69
:1020600042C083EE4DC08091740282FF38C0F5CF2C
:102070008091740282FD33C08091750280FD31C071
:10208000ECCF8091750281FF32C08091740284FD93
:102090002AC087EE35C08091740283FF26C0F5CF39
:1020A0008091740283FD21C08091750281FD1FC063
:1020B000ECCF8091740285FD1CC01DC0809174021C
:1020C00085FD19C016C08091740286FD16C017C028
:1020D0008091740286FD13C010C089E311C082EEA6
:1020E0000FC080EE0DC080E00BC086EE09C084EE0C
:1020F00007C089E205C085E303C08AE201C081E32D
:1021000090E008959091740292FF0DC0282F2871DD
:10211000283019F4877F846006C0282F247124306A
:1021200011F48B7F886093FF0DC0282F2871283110
:1021300019F4877E846106C0282F2471243111F49C
:102140008B7E88612091750220FF0DC0382F387179
:10215000383019F4877F816006C0382F31713130F3
:1021600011F48E7F886021FF0DC0282F287128313F
:1021700019F4877E816106C0282F2171213111F465
:102180008E7E886194FD877E089510927002109271
:1021900071021092720210927302089580E0089505
:1021A0000C94360D0E944C128FEB9DE50197F1F7D0
:1021B00000C000000E944C1280E00E940C1180FFC1
:1021C00004C00E94D0100C94B21908950C94D2103F
:1021D0000E943C0D811102C00E94E40D0E94470D37
:1021E00080933A020E944F0D90937502809374027F
:1021F0000E94E6100E944B0D682F70E080E090E096
:102200000E9458076091D2017091D3018091D4014E
:102210009091D5010C949007E82FF0E0ED57FD4F19
:1022200080810895089580EA8A95F1F7089500C0A5
:1022300008950C94131108950C941B110C941C1107
:102240000C941B110C9420110C941B11FF920F93F2
:102250001F93CF93DF9300D000D000D0CDB7DEB76F
:102260000E94D71260918F028823E9F186E0F82E50
:102270008E010F5F1F4FF8018F2D11928A95E9F79C
:10228000862F90E0B8018D579D4F0E94021388233E
:1022900089F08091760290E046E050E0B8018D57D9
:1022A0009D4F0E94CF2021E020933B02892B61F4B7
:1022B00010E016C080913B028823D1F3F8011192FF
:1022C000FA94E9F710923B02A0917602B0E0AD5784
:1022D000BD4F86E0F80101900D928A95E1F711E07B
:1022E0000E94D4020DC070E06D577D4F8091760240
:1022F00090E08D579D4F0E946B020E94241110E0C8
:10230000812F26960FB6F894DEBF0FBECDBFDF91AA
:10231000CF911F910F91FF900895F894E82FE295C7
:10232000EF70F0E031A1282F2F7081E090E001C024
:10233000880F2A95EAF7982F9095932391A392A15D
:10234000892B82A3789408950F931F93CF93DF93E3
:10235000C3E8D1E089918F3F11F00E948D1181E097
:10236000C938D807B9F7CCE7D1E003E811E0899183
:102370008F3F11F00E948D110C171D07C1F7DF91DF
:10238000CF911F910F910895CF92DF92EF92FF921C
:102390000F931F93CF93DF938C01C62FD0E0CE0114
:1023A0008D579E4F7C01FC0190819F3F09F447C0EF
:1023B000D62EF894E92FE295EF70F0E081A19F709E
:1023C00021E030E001C0220F9A95EAF7822B81A329
:1023D00082A12095282322A378940E941711ECE76C
:1023E000F1E043E851E031E0C12C21912F3F89F029
:1023F000A22FA295AF70B0E090968C9190E02F70D4
:1024000002C0959587952A95E2F780FD02C0832F3B
:1024100001C080E0C82A330F4E175F0731F7F7017C
:1024200080818F3F11F00E948D1161E0C11001C0C9
:1024300060E08D2D0E941911C00FD11FC882DF915D
:10244000CF911F910F91FF90EF90DF90CF90089563
:102450008091040180910401811102C096E001C0C5
:1024600090E090938F0286E0891B809376020E9411
:10247000A4118CE0E3E8F2E0DF01982F1D929A9519
:10248000E9F7E7E7F2E0DF011D928A95E9F786E0D8
:102490000E94A0120C94D202EF92FF920F931F930E
:1024A000CF93DF93CDB7DEB72C970FB6F894DEBF8E
:1024B0000FBECDBF8E010F5F1F4F8CE0F801119250
:1024C0008A95E9F7F12C6F2DC8010E94C411F3948D
:1024D000F6E0FF12F8CF4CE050E0B80187E792E059
:1024E0000E94CF207C0121E0892B09F420E0E11437
:1024F000F10441F08CE0F801A7E7B2E001900D9201
:102500008A95E1F760918F0270E06D577D4F46E04C
:1025100087E792E00E94A112EF2819F40E94261189
:1025200002C081E090E02C960FB6F894DEBF0FBE9B
:10253000CDBFDF91CF911F910F91FF90EF90089544
:102540000895FF920F931F93CF93DF938C01F62E84
:10255000D72FC42F222349F081E080933E020E94AE
:10256000651990933D0280933C0280913E0288233E
:10257000C1F080913C0290913D020E947D19039729
:1025800080F0EF2DFD2FD8014C2F50E0CD01801BA6
:10259000910B841795071CF48D918193F7CF1092BE
:1025A0003E02DF91CF911F910F91FF90089580918E
:1025B000410281110DC00E949420811102C082E06D
:1025C00001C081E080934102823011F40E948F208B
:1025D00081E090914102913009F080E008950C94DF
:1025E000D7120E94EF12809304010E94D71281112A
:1025F0000C94570208950E94D712811102C00C94C6
:10260000530208950F931F93CF93DF93EC018B0137
:10261000809142028A3038F4B801CE010E945902FA
:1026200081111DC00AC080913F02909140020E941A
:102630007D19843F914080F715C0809142028F3F01
:1026400019F08F5F80934202809142028A3060F0DD
:102650000E9465199093400280933F0203C010923C
:10266000420202C080E001C081E0DF91CF911F9162
:102670000F9108950E94551B0E94260E0C94611B19
:102680000E94651B0E94BC0E0C947F1B0E940319C4
:102690000E943C1B0E94140E0E943A130E94401399
:1026A0000E941E0EFBCF8091490280FF06C0609100
:1026B0000A0170E0660F771F26C081FF04C0609199
:1026C0000A0184E005C082FF07C060910A0188E02A
:1026D000689FB001112417C0909148029923D1F04E
:1026E00060910901961788F720910A0188E0289FD8
:1026F00090011124929FA001939F500D112470E02E
:10270000CA010E94A1206038710540F4611571056D
:1027100019F406C068E070E0862F08958FE70895E9
:1027200081E008958091490280FF08C06091060110
:1027300070E0759567957595679521C081FF06C016
:102740006091060170E07595679519C082FF04C01D
:102750006091060170E010C090914702992399F0B2
:10276000609105019617A0F780910601899FC0012D
:10277000112470E00E94A1206038710540F46115B9
:10278000710519F406C061E070E0862F08958FE7A7
:10279000089581E008958D3E21F40E9453138195A0
:1027A00004C08E3E29F40E94531380934D02089575
:1027B0008F3E21F40E945313819504C0803F29F479
:1027C0000E94531380934C020895893F19F40E948C
:1027D000921305C08A3F31F40E9492138195809331
:1027E0004E0208958B3F21F40E949213819504C0FC
:1027F0008C3F29F40E94921380934F0208959FE02A
:10280000980F983078F421E030E0A90102C0440F1D
:10281000551F9A95E2F7CA0190914B02892B80933C
:102820004B0208958D3F21F48091490281600BC0D5
:102830008E3F21F480914902826005C08F3F29F4C8
:102840008091490284608093490208958D3E39F455
:1028500090914D0297FF35C010924D0259C08E3EA7
:1028600029F490914D021916BCF32BC090914C02A3
:102870008F3E29F497FF25C010924C0249C0803F3B
:1028800019F41916CCF31DC090914E02893F29F41A
:102890001916BCF410924E023BC08A3F19F497FF00
:1028A00010C0F8CF8B3F39F490914F0297FF09C0C9
:1028B00010924F022DC08C3F21F490914F021916B7
:1028C000BCF39FE0980F983080F421E030E0A9013C
:1028D00002C0440F551F9A95E2F7CA018095909166
:1028E0004B02892380934B0213C08D3F21F48091CA
:1028F00049028E7F0BC08E3F21F4809149028D7F6B
:1029000005C08F3F29F4809149028B7F8093490253
:1029100080914C02811106C080914D02811102C04C
:102920001092480280914E02811106C080914F02A0
:10293000811102C01092470208950E9465192091EA
:102940004C02211104C020914D02222321F09093CA
:1029500046028093450220914E02211104C020912D
:102960004F02222321F090934402809343028AE491
:1029700092E00C944318EF92FF920F931F93CF9322
:10298000DF9300D000D000D0CDB7DEB786E0EAE418
:10299000F2E0DE01119601900D928A95E1F7E09048
:1029A0004C02F0904D0200914E0210914F02109295
:1029B0004C0210924D0210924E0210924F02E11002
:1029C00003C0FF2009F45DC080914502909146024A
:1029D0000E947D19AC0190914802992339F0209111
:1029E0000B0130E02417350758F04BC020910C0143
:1029F0008AE0289F900111242417350718F041C060
:102A00009F3F19F09F5F90934802EE2061F00E9473
:102A100053131E1414F09FEF01C091E0989F902D66
:102A2000112490934C02FF2061F00E9453131F1455
:102A300014F09FEF01C091E0989F902D1124909386
:102A40004D0230914C023323E1F020914D022223BC
:102A5000C1F045EB3403C0011124992319F0909380
:102A60004C0203C081E080934C0235EB2303C0018C
:102A70001124992319F090934D0203C081E08093B3
:102A80004D02011103C0112309F45DC0809143027E
:102A9000909144020E947D19AC01909147029923C4
:102AA00039F02091070130E02417350758F04BC06A
:102AB000209108018AE0289F9001112424173507EE
:102AC00018F041C09F3F19F09F5F90934702002389
:102AD00061F00E949213101614F09FEF01C091E074
:102AE000989F902D112490934E02112361F00E9423
:102AF0009213111614F09FEF01C091E0989F902D52
:102B0000112490934F0230914E023323E1F0209133
:102B10004F022223C1F045EB3403C0011124992355
:102B200019F090934E0203C081E080934E0235EB82
:102B30002303C0011124992319F090934F0203C07D
:102B400081E080934F0280914C0281110BC08091F3
:102B50004D02811107C080914E02811103C0809106
:102B60004F0281110E949D14EB82FC820D831E8313
:102B700086E0FE013196AAE4B2E001900D928A95BA
:102B8000E1F726960FB6F894DEBF0FBECDBFDF91FA
:102B9000CF911F910F91FF90EF900895EAE4F2E03A
:102BA00086E0DF011D928A95E9F7109248021092A3
:102BB00047021092490208950895CF93DF93EC01E4
:102BC000FB018281882309F43CC1C430FDE5DF07A5
:102BD00060F4CB3F9CE5D90788F49E0122503C4528
:102BE0002431310508F02EC109C0C236EDE5DE07FB
:102BF00029F0C63AFDE5DF0709F024C10E944F0D18
:102C00009093750280937402C1318CE5D80709F462
:102C1000C6C008F042C0C930ECE5DE0709F49BC02D
:102C200000F5C5308CE5D80709F485C078F4C330C9
:102C3000ECE5DE0709F478C008F07AC0C230DC4564
:102C400009F0F5C0809174028160EFC0C7309CE547
:102C5000D90709F478C008F07AC0809174028061C5
:102C6000E4C0CD30FCE5DF0709F487C058F4CB3071
:102C70009CE5D90709F479C008F07BC08091740203
:102C800088606FC0CF30FCE5DF0709F480C008F032
:102C900082C080917402877FC8C0CE3F9CE5D9076F
:102CA00009F471C000F5C531FCE5DF0709F485C002
:102CB00068F4C3319CE5D90709F475C008F095C0E4
:102CC0000E940007809174028F77AFC0CC3FFCE573
:102CD000DF07A9F108F054C0CB3FDC4509F0A7C0DD
:102CE0008091750240C0C230EDE5DE0709F489C06D
:102CF00058F4C1158DE5D80709F45AC008F069C029
:102D00008091750282602FC0C236EDE5DE0709F4BE
:102D10007CC0C63AFDE5DF0709F481C0C330DD455C
:102D200009F085C080E06EC08091740282607DC031
:102D30008091740216C080917402886076C0809180
:102D4000750282604FC08091740280626EC0809173
:102D5000740280646AC00E940007809174028068D7
:102D600064C0846062C081603DC0809174028E7FC7
:102D70005CC0809174028D7F58C08091740216C02F
:102D80008091750218C0809175028D7F2BC0809153
:102D900074028F7E4AC0809174028F7D46C08091FC
:102DA00074028F7B42C080917402877F8B7F3DC00D
:102DB000809175028D7F8E7F15C08091740282FB99
:102DC000222720F991E0922790FB82F990FB83F96A
:102DD0002CC080917502982F909591708E7F892BD1
:102DE00090FB81F98093750222C00E9400078091B8
:102DF000740287FB222720F991E0922790FB87F944
:102E000014C081E00E94E60D12C08091740284FB20
:102E1000222720F991E0922790FB84F906C0809147
:102E20007402982F909590FB80F9809374028091A2
:102E30007402909175020E94600D0E94000780E06C
:102E400001C081E0DF91CF910895CF93DF93863168
:102E50009C4541F5EB010E94530C982F8A812091EB
:102E6000020130910301882379F09A7A81E009F414
:102E700080E080935002911102C069E201C065E3D5
:102E8000C9010E94BF180AC080915002811102C07E
:102E900069E201C065E3C9010E94C1180E94950C56
:102EA00080E001C081E0DF91CF9108950F931F93DF
:102EB000CF93DF93C42FD22FFC0182818823C9F0E6
:102EC000409353020E9465199093520280935102DD
:102ED00080E28C0F883008F057C0C77081E001C0D5
:102EE000880FCA95EAF7DF91CF911F910F910C944B
:102EF0005D0480915302481330C08091510290913B
:102F000052020E947D19883C910538F510E21D0F90
:102F1000CD17B9F080E28C0F883040F4C77081E0A3
:102F200001C0880FCA95EAF70E946404183028F59A
:102F300081E09D2F977001C0880F9A95EAF70E9453
:102F40005D04802F0E9454041830F0F4D77081E0A3
:102F500001C0880FDA95EAF70AC080E28C0F88304A
:102F600098F4C77081E001C0880FCA95EAF7DF9135
:102F7000CF911F910F910C946404802FDF91CF911A
:102F80001F910F910C945404DF91CF911F910F91D9
:102F900008950F939C01CB01243F4CE5340731F198
:102FA00088F4293DFCE53F07D9F02A3D4CE534077C
:102FB00079F1283D3C45A9F506E221EE41EE68EDA8
:102FC0007CE52BC0263FFCE53F07E1F0A8F0273F5A
:102FD0003C4539F507E225EE46EE67EF7CE51DC07E
:102FE00007E225EE45EE69ED7CE517C006E221EE2D
:102FF00040EE64EF7CE511C007E225EE44EE65EF9C
:103000007CE50BC006E221EE42EE66EF7CE505C0F2
:1030100008E221E045EE6AED7CE50E94561780E06B
:1030200008C0FC018281882319F01092530201C06C
:1030300081E00F91089590938B0180938A01089508
:1030400090935A028093590208950E94D7128111D9
:1030500003C0809154020895E0915902F0915A0200
:10306000309721F00190F081E02D099480E00895DF
:10307000E0915902F0915A02309721F00280F381D9
:10308000E02D09940895E0915902F0915A02309789
:1030900039F022E0DC012C930480F581E02D0994C5
:1030A000089520915702309158022817390771F07E
:1030B0009093580280935702E0915902F0915A027E
:1030C000309721F00680F781E02D09940895209132
:1030D0005502309156022817390771F09093560225
:1030E00080935502E0915902F0915A02309721F0F5
:1030F0000084F185E02D09940895FC01329697E053
:1031000080E0915029F021912223D9F38F5FF9CFEC
:103110000895662349F0FC013296089621916217C2
:1031200029F0E817F907D1F780E0089581E00895C4
:103130009C01FC0132969FEF80E04191461789F097
:103140009F3F19F4411101C0982F8F5F8630A9F776
:103150009F3F39F0F901E90FF11D97FDFA95628360
:10316000089508959C012A5F3F4FFC014281461358
:1031700001C01282019682179307B9F708950C9443
:1031800098180C94B218029626E0FC0111922A9528
:10319000E9F7089508950C94CA1883E080935B02C0
:1031A0000C94CB18811102C081E001C082E08093B1
:1031B0005B020C94CB180C94D21881E080935B02D4
:1031C0000C94CB180C94DD1808950C94E4180C940E
:1031D000E5180C94E4180C94E4180C94E418CF93BC
:1031E0000E94EB180E944C120E94E918C0E08C2F3C
:1031F0000E940C11811104C0CF5FCC30C1F701C017
:1032000081E0CF91089508951F920F920FB60F920B
:1032100011248F939F93AF93BF9380915C02811190
:1032200013C08091900290919102A0919202B0916E
:1032300093024196A11DB11D80939002909391023B
:10324000A0939202B0939302BF91AF919F918F91FF
:103250000F900FBE0F901F901895809198028430A8
:1032600031F10E94380310925C0220E488E190E082
:103270000FB6F894A895809360000FBE209360006D
:1032800083B7817F846083BF83B7816083BF789475
:10329000889583B78E7F83BF0FB6F894A8958091E9
:1032A0006000886180936000109260000FBE0895F6
:1032B0000E9400070C943C0382E084BD93E095BD1E
:1032C0009AEF97BD80936E0008952FB7F894809180
:1032D000900290919102A0919202B09193022FBF1F
:1032E00008952FB7F89460919002709191028091A7
:1032F0009202909193022FBF08959C014FB7F894CA
:103300008091900290919102A0919202B0919302CB
:103310004FBF821B930B089578941F920F920FB6A4
:103320000F9211248F939F93AF93BF93809190023C
:1033300090919102A0919202B09193020196A11DE9
:10334000B11D8093900290939102A0939202B0934A
:103350009302BF91AF919F918F910F900FBE0F90ED
:103360001F90189587E797E79093010880930008CE
:103370009AE088E10FB6F894A895809360000FBE9C
:1033800090936000FFCF809168020895089522E035
:103390002093E9002FEF3091E800215035FD06C061
:1033A00035ED3A95F1F700002111F5CF2091E800B5
:1033B00025FF0BC040E050E066E070E00E94F11B8A
:1033C0008091E8008E778093E8000895CF93DF9393
:1033D00021E02093E9002FEF3091E800215035FDE6
:1033E00006C035ED3A95F1F700002111F5CF209197
:1033F000E80025FF14C0EC0140E050E068E070E018
:103400000E94F11B8091E8008E778093E80088E0AD
:10341000FE01A0E6B2E001900D928A95E1F7DF91FE
:10342000CF91089580935D0270935F0260935E0276
:1034300080919802843001F582E08093E9008FEF5B
:103440009091E800815095FD06C095ED9A95F1F7B1
:1034500000008111F5CF8091E80085FF0DC040E0AC
:1034600050E063E070E08DE592E00E94F11B8091F6
:10347000E8008E778093E8000895BC0184E00C9406
:10348000121ABC0183E00C94121A809197028111E8
:1034900009C00E94821D0E94DF1D8091E2008460AD
:1034A0008093E20008951092970208950C94E21818
:1034B0006091940281E0611101C080E00C94CD180C
:1034C0009091980281E0943009F080E0609194023C
:1034D0000C94D21842E061EC81E00E94FB1C42E2B5
:1034E00061EC82E00E94FB1C9091980281E0943094
:1034F00009F080E0609194020C94DB1880919A02AC
:10350000833009F461C030F4813071F0823009F405
:103510009AC008958A3009F486C08B3009F46CC0D3
:10352000893009F0A8C020C080919902813A09F041
:10353000A2C08091E800877F8093E80080919D027F
:1035400090919E02892B21F468E080E692E003C00E
:1035500060E080E090E070E00E943C1C8091E80018
:103560008B778093E800089580919902813209F069
:1035700082C080919D0290919E02029708F07BC0CC
:103580008091E800877F8093E8008091E80082FDC9
:1035900005C0809198028111F8CF6DC02091F30091
:1035A0008091F20090E0922B029731F48091F1002B
:1035B000813011F0863021F48091F100809368020F
:1035C0008091E8008B7753C080919902813A09F08D
:1035D00052C080919D0290919E02892B09F04BC0B0
:1035E0008091E800877F8093E8008091E80080FF69
:1035F000FCCF8091190136C0809199028132D9F5B2
:1036000080919D0290919E02892BA9F58091E800FE
:10361000877F8093E8000E94301D80919B028093F9
:1036200019010C94000780919902813221F5809153
:10363000E800877F8093E8000E94301D80919C0203
:1036400080936902089580919902813AA1F4809152
:10365000E800877F8093E8008091E80080FFFCCF3E
:10366000809169028093F1008091E8008E778093C9
:10367000E8000C94301D089584B7877F84BF0FB68F
:10368000F894A89580916000886180936000109202
:1036900060000FBE90E080E80FB6F8948093610060
:1036A000909361000FBE0C94DD180E94821D0E9451
:1036B000DF1DE2EEF0E080818460808378940C94DA
:1036C00074208DE091E00C94201880919802853050
:1036D000A9F480919802853079F40E942D19809187
:1036E00096028823B1F30E94EF18882391F30E9479
:1036F000DB1B0E940007EDCF0C9458190895089524
:103700000C94821B292F332723303105C9F060F434
:103710002130310581F02230310509F044C08BE3BE
:1037200090E020EC31E043C021323105E1F022325B
:10373000310549F138C082E190E02BEF31E037C02C
:1037400099278130910549F028F0029761F5E0E86A
:10375000F1E005C0ECEBF1E002C0E8EAF1E08491B1
:1037600090E09F0124C06115710541F06130710541
:10377000D1F489E090E02BEE31E019C089E090E0CF
:1037800022ED31E014C06115710541F06130710521
:1037900051F48BE790E02DE032E009C080E490E046
:1037A00028E832E004C080E090E020E030E0FA0158
:1037B00031832083089580E189BD82E189BD09B408
:1037C00000FEFDCF8091D8008F7D8093D80080913E
:1037D000E00082608093E0008091E00081FDFCCFFA
:1037E0000895CF92DF92EF92FF920F931F93CF93A2
:1037F000DF93EC018B017A010E944F1D811133C0D0
:10380000E114F10439F0F70180819181081B190B53
:10381000C80FD91FC12CD12C0115110519F18091A8
:10382000E80085FD16C08091E8008E778093E8005F
:10383000E114F10449F0F70180819181C80ED91E8D
:10384000D182C08285E00FC00E944F1D882321F3E2
:103850000AC089918093F10001501109FFEFCF1A3E
:10386000DF0ADACF80E0DF91CF911F910F91FF90B7
:10387000EF90DF90CF90089520919F023091A002A9
:103880002617370748F06115710539F42091E800D3
:103890002E772093E80001C0B901FC0120E06115FA
:1038A000710579F1809198028823F1F18530F1F169
:1038B0008091E80083FD3CC08091E80082FD2EC02D
:1038C0008091E80080FFEBCF2091F3008091F2001F
:1038D00090E0922B6115710551F08830910538F414
:1038E00021912093F100615071090196F3CF21E0FD
:1038F000089709F020E08091E8008E778093E80037
:10390000CECF2111CFCF0AC080919802882361F0D9
:10391000853061F08091E80083FD0AC08091E80065
:1039200082FFF2CF80E0089582E0089583E0089559
:1039300081E0089520919F023091A0022617370759
:1039400048F06115710539F42091E8002E77209335
:10395000E80001C0B901FC0120E06115710591F199
:1039600080919802882309F440C0853009F43FC053
:103970008091E80083FD3DC08091E80082FD2FC06A
:103980008091E80080FFE9CF2091F3008091F20060
:1039900090E0922B6115710559F08830910540F443
:1039A00024912093F1003196615071090196F2CF74
:1039B00021E0089709F020E08091E8008E7780935D
:1039C000E800CBCF2111CCCF0AC080919802882388
:1039D00061F0853061F08091E80083FD0AC080913C
:1039E000E80082FFF2CF80E0089582E0089583E04E
:1039F000089581E00895982F973068F59093E90035
:103A0000981739F07091EC002091ED005091F00082
:103A100003C0242F762F50E021FD02C09F5FECCF22
:103A20003091EB003E7F3093EB003091ED003D7F15
:103A30003093ED003091EB0031603093EB007093E8
:103A4000EC002093ED005093F0002091EE0027FD54
:103A5000E5CF80E008958F708093E90081E00895BC
:103A60008091990287FF11C08091E80082FD05C016
:103A7000809198028111F8CF11C08091E8008B7776
:103A80000BC080919802882349F08091E80080FF64
:103A9000F8CF8091E8008E778093E8000895209118
:103AA000E4003091E50095E64091EC00842F8170B0
:103AB00040FF23C08091E80080FD1DC080919802E6
:103AC000882399F0853099F08091EB0085FD11C035
:103AD0004091E4005091E5002417350729F39150F7
:103AE00011F09A01E1CF84E0089582E0089583E027
:103AF000089581E0089580E008954091E80042FF34
:103B0000DDCF08950E94F01D0E94F81DE0EEF0E068
:103B1000808181608083E8EDF0E080818F77808311
:103B200019BCA7EDB0E08C918E7F8C9380818F7E45
:103B300080831092970208950F931F93CF93DF9382
:103B40000E94F01D0E94F81DC8EDD0E088818F779B
:103B5000888388818068888388818F7D888319BC69
:103B6000109298021092940210929602109295026E
:103B700000EE10E0F80180818B7F80838881816076
:103B8000888342E060E080E00E94FB1CE1EEF0E010
:103B900080818E7F8083E2EEF0E08081816080838F
:103BA000808188608083F80180818E7F8083888116
:103BB00080618883DF91CF911F910F910895E8ED87
:103BC000F0E080818F7E8083E7EDF0E0808181608E
:103BD000808384E082BF81E0809397020C949C1DD7
:103BE000E8EDF0E080818E7F80831092E2000895FE
:103BF0001092DA001092E10008951F920F920FB612
:103C00000F9211242F933F934F935F936F937F9362
:103C10008F939F93AF93BF93EF93FF938091E100B6
:103C200082FF0BC08091E20082FF07C08091E1001B
:103C30008B7F8093E1000E9473208091DA0080FFE7
:103C40001FC08091D80080FF1BC08091DA008E7F5A
:103C50008093DA008091D90080FF0DC080E189BD9A
:103C600082E189BD09B400FEFDCF81E08093980216
:103C70000E94451A05C019BC109298020E94531A5E
:103C80008091E10080FF19C08091E20080FF15C0A3
:103C90008091E2008E7F8093E2008091E20080615B
:103CA0008093E2008091D80080628093D80019BC94
:103CB00085E0809398020E94581A8091E10084FF69
:103CC00030C08091E20084FF2CC080E189BD82E198
:103CD00089BD09B400FEFDCF8091D8008F7D80930F
:103CE000D8008091E1008F7E8093E1008091E20016
:103CF0008F7E8093E2008091E20081608093E200F9
:103D000080919402882311F084E007C08091E30041
:103D100087FD02C081E001C083E0809398020E9489
:103D2000601A8091E10083FF29C08091E20083FF47
:103D300025C08091E100877F8093E10082E080933D
:103D40009802109294028091E1008E7F8093E100AE
:103D50008091E2008E7F8093E2008091E20080619A
:103D60008093E20042E060E080E00E94FB1C8091D2
:103D7000F00088608093F0000E94561AFF91EF9146
:103D8000BF91AF919F918F917F916F915F914F9173
:103D90003F912F910F900FBE0F901F9018951F927B
:103DA0000F920FB60F9211242F933F934F935F936F
:103DB0006F937F938F939F93AF93BF93CF93DF9333
:103DC000EF93FF93C091E900CF708091EC00D82F62
:103DD000D17080FDD0E81092E9008091F000877FDB
:103DE0008093F00078940E94131F1092E900809154
:103DF000F00088608093F000CD2BCF70C093E90075
:103E0000FF91EF91DF91CF91BF91AF919F918F91F2
:103E10007F916F915F914F913F912F910F900FBEC6
:103E20000F901F9018951F93CF93DF93CDB7DEB7F8
:103E3000AA970FB6F894DEBF0FBECDBFE9E9F2E056
:103E40008091F100819322E0E13AF207C9F70E94E4
:103E50007E1A8091E80083FF2EC180919902909193
:103E60009A02492F50E04A30510508F024C1FA0166
:103E7000EE59FF4F0C94B520803821F0823809F0BC
:103E80001AC108C08091950290919602992389F0F9
:103E900082600FC080919D028F70873008F00BC147
:103EA0008093E9008091EB0085FB882780F91092D0
:103EB000E9009091E800977F9093E8008093F100EB
:103EC0001092F100D1C0282F2D7F09F0F4C0882373
:103ED00019F0823061F0EFC080919B02813009F0CF
:103EE000EAC0933009F080E0809396022EC0809162
:103EF0009B0281112AC080919D028F702FEF280FA5
:103F0000263008F0D8C08093E9002091EB0020FF14
:103F10001CC0933021F48091EB00806214C090911A
:103F2000EB0090619093EB0021E030E0A90102C02A
:103F3000440F551F8A95E2F74093EA001092EA0079
:103F40008091EB0088608093EB001092E9008091F3
:103F5000E800877F8093E8000E94301DACC081118B
:103F6000AAC010919B021F778091E3008078812B7B
:103F70008093E3008091E800877F8093E8000E94AF
:103F8000301D8091E80080FFFCCF8091E3008068C5
:103F90008093E300111102C082E001C083E08093AE
:103FA000980289C08058823008F085C080919B02B9
:103FB00090919C028C3D53E0950779F583E08A83CC
:103FC0008AE289834FB7F894DE01139620E03EE041
:103FD00051E2E32FF0E050935700E49120FF03C03B
:103FE000E295EF703F5FEF708E2F90E0EA3010F0B7
:103FF000C79601C0C0968D939D932F5F243149F7DA
:104000004FBF8091E800877F8093E8006AE270E00C
:10401000CE0101960E943C1C16C060919D027091D9
:104020009E02AE014F5F5F4F0E94801BBC01892B37
:1040300009F441C09091E800977F9093E80089814E
:104040009A810E949A1C8091E8008B778093E80007
:1040500032C0803881F58091E800877F8093E80046
:10406000809194028093F1008091E8008E7772CF66
:10407000811121C080919B0290919C029927029707
:10408000D4F48091E800877F8093E80080919B02C0
:10409000809394020E94301D80919402811106C089
:1040A0008091E30087FD02C081E001C084E080933D
:1040B00098020E946A1A8091E80083FF0AC08091EA
:1040C000E800877F8093E8008091EB008062809316
:1040D000EB00AA960FB6F894DEBF0FBECDBFDF91FE
:1040E000CF911F9108950895CF93809198028823CE
:1040F000A1F0C091E900CF709091EC00892F817000
:1041000090FD80E8C82B1092E9008091E80083FDC3
:104110000E94131FCF70C093E900CF9108950E94B1
:10412000821D109298020895E8EDF0E08081806190
:1041300080838AE18A95F1F700C08091D90081706F
:10414000089597FB072E16F4009407D077FD09D049
:104150000E94BB2007FC05D03EF4909581959F4FAF
:104160000895709561957F4F0895EE0FFF1F05909C
:10417000F491E02D0994AA1BBB1B51E107C0AA1FB3
:10418000BB1FA617B70710F0A61BB70B881F991FF8
:104190005A95A9F780959095BC01CD010895FB0132
:1041A000DC0104C08D910190801921F441505040F0
:1041B000C8F7881B990B0895F999FECF92BD81BD70
:1041C000F89A992780B50895A8E1B0E042E050E060
:1041D0000C941021262FF999FECF92BD81BDF89A3B
:1041E000019700B4021639F01FBA20BD0FB6F8943B
:1041F000FA9AF99A0FBE08950396272F0E94EB2092
:104200000E94EA20252F0E94EB20242F0C94EB2003
:104210000196272F0E94EB200C94EA20DC01CB01B1
:10422000FC01F999FECF06C0F2BDE1BDF89A3196C6
:1042300000B40D9241505040B8F70895F894FFCF64
:10424000C8001C0201280850011E0A1401C319E607
:1042500019C719411A3D1AC61901E200E900EA001E
:10426000B500B600B700CD008301CC008A019201F1
:1042700094012102230224022502260227022A0297
:10428000B300B4006F007000818283E200E900EAAD
:1042900000B500B600B700CD008301CC008A0192C2
:1042A0000194012102230224022502260227022A68
:1042B00002B300B4006F007000818283946697C6D9
:0A42C000F4F5F631323334353600E0
:00000001FF
